S01700006F70656E626C745F7333326B3131382E73726563DD
S113000000580020091D0000030B0000030B000032
S113001000000000000000000000000000000000DC
S1130020000000000000000000000000030B0000BE
S11300300000000000000000030B0000030B0000A0
S1130040030B0000030B0000030B0000030B000074
S1130050030B0000030B0000030B0000030B000064
S1130060030B0000030B0000030B0000030B000054
S1130070030B0000030B0000030B0000030B000044
S1130080030B0000030B0000030B0000030B000034
S1130090030B0000030B0000030B0000030B000024
S11300A0030B0000030B0000030B0000030B000014
S11300B0030B0000030B0000030B0000030B000004
S1130400FFFFFFFFFFFFFFFFFFFFFFFFFE7FFFFF79
S113041008B4024B9C4608BC6047C046C10000209B
S11304200020C04399490860994908607047F2B5B3
S1130430070014000125974ED8203058DC2171584C
S11304404018401EC01B0099491E884200D2002556
S11304502800C0B201280CD1380000F063FAFF284C
S113046006D000983818401E00F05CFAFF2800D12E
S113047000252800C0B2012814D1380A802149007F
S1130480484322003168884206D1009B39008048E5
S113049000F002F9050005E0009B39007B4800F0FC
S11304A0FBF805002800C0B2F2BDF8B504000F0047
S11304B001267849D8228A58DC23C9585118491E84
S11304C0091B7A1E914200D200263100C9B20129CB
S11304D010D1200000F026FA0500E019401E00F0BB
S11304E021FA2900C9B2FF2903D00100C9B2FF29AA
S11304F000D100263100C9B2012906D10100C9B2D8
S11305002800C0B200F091F906003000C0B2F2BD7C
S113051080B50120002100915D490A680023DB4376
S11305209A422CD00200D2B2012A28D100984A68FB
S11305308018009000988A68801800900098CA6813
S11305408018009000980A698018009000984A6901
S11305508018009000988A69801800900098C969F2
S1130560401800900098C14300910098401C0090EE
S11305706A46042147480068C030FFF758FFC0B2FC
S113058002BD10B5012000210B00424A1468246802
S11305901B191468241D24681B1914680834246862
S11305A01B1914680C3424681B191468103424684B
S11305B01B191468143424681B191468183424682B
S11305C01B191268C03212689A18002A00D0080059
S11305D0C0B210BD38B501240025ED432C48016894
S11305E0A94204D000F0A6F8002800D1002420007D
S11305F0C0B2012808D125480168A94204D000F0FE
S113060099F8002800D100242000C0B232BD21484E
S11306100068704710B50124CAB2002A00D0002433
S11306202200D2B2012A08D102688A4205D00160B0
S113063080225200001D00F0DBF92000C0B210BD82
S1130640F8B504000E00002738001148844202D196
S11306500E4C25000EE00F490A68964203D10400AF
S11306600E68250006E02500200000F063F800284D
S113067000D13D00002D06D031002000FFF7CAFF55
S1130680002800D13D002800F2BD00000C310020FC
S1130690103200204C1B0000FEB504000E001700B1
S11306A00125300A80214900484300902068002138
S11306B0C943884206D100992000FFF7ABFF002808
S11306C000D100252800C0B201280BD12068009970
S11306D0884207D000992000FFF7B2FF0400002CE5
S11306E000D100252800C0B2012820D12068301A8A
S11306F02018061D00F091F980204000211D711A78
S1130700814208D3009909182000FFF799FF0400DB
S1130710002C0BD0261D38783070761C7F1C029874
S1130720401E029002980028E4D100E00025280031
S1130730C0B2FEBDF1B582B001240820694608703C
S11307400298006800F0EEF8FF2800D10024200091
S1130750C0B2012864D10020019012E0491C0A00B3
S11307606B461B78D2B29A4208D20A00D2B2AA5C73
S11307700B00DBB2F35C9A42F0D004000198401CF9
S11307800190802040006946097800F060F90199E1
S1130790814245D20298006801996A461278514311
S11307A04518029801996A46127851434018061D6B
S11307B000F033F96E4F3878000630D57020387069
S11307C007206C4908702800000C6B490870280A3F
S11307D06A49087028006A490870307869490870C5
S11307E0707869490870B07868490870F078684989
S11307F00870307967490870707967490870B07972
S113080066490870F07966490870FFF701FE387888
S113081071210140002906D1002001009FE7002436
S11308202000C0B2FEBD0024FAE7F2B582B0012474
S11308306946097A0200D2B2914200D20024210012
S1130840C9B2012904D16946097A132900D30024C5
S11308502100C9B2012962D1070000E07F1C68466B
S1130860007A3900C9B2884259D300F0D6F84D480D
S11308703900C9B20C225143415801913900C9B21F
S11308800C2251434018406801990022D2439142FE
S11308900FD000280DD001994905490D00290AD12E
S11308A04105490D002908D1C00A69460870002590
S11308B01BE0002433E0002431E000242FE0702109
S11308C0317009212B4A11700100090C2A4A117058
S11308D0010A2A4A11702A490870FFF799FD3078F5
S11308E071210140002915D16D1C28006946097841
S11308F0C0B288420FD200F090F801982900C9B222
S11309008022120151434018194E31780906D6D479
S1130910002400E000242000C0B200289ED1200062
S1130920C0B2FEBD70B50400FF25002600E0761CB1
S11309303000C0B2132818D200F06FF81948310003
S1130940C9B20C22514341588C42F0D33100C9B290
S11309500C22514341583200D2B20C235A4380181E
S1130960406808188442E2D235002800C0B270BD45
S11309700000024007000240060002400500024059
S11309800400024008000240090002400A0002403C
S11309900B0002400C0002400D0002400E00024019
S11309A00F0002404C1B000080B500F0ABF801BD05
S11309B080B500F0B7F8002814D000F0C5F800287E
S11309C010D000F005F900F064F900F0AFF8064922
S11309D001400648016000F097F800F0A7F8001DF8
S11309E00068804701BD000080FFFF1F08ED00E0A4
S11309F070B514000D00060005E0287830706D1CF9
S1130A00761C00F00AF82000441E80B20028F4D1BD
S1130A1070BD80B500F0A6F801BD80B500F0A7F860
S1130A2001BDF446002804D4494200F013F84042C2
S1130A3060474042002905D45FD000F00BF84042E3
S1130A4049426047494200F005F84942604703467D
S1130A500B43E6D40022030A8B420BD203098B42D8
S1130A6019D243088B422ED2411A00D20146524178
S1130A7010467047FF2209023FD012068B4205D36D
S1130A80121209028B4201D31212090203098B428A
S1130A9019D300E0090AC3098B4201D3CB01C01A60
S1130AA0524183098B4201D38B01C01A524143093D
S1130AB08B4201D34B01C01A524103098B4201D32B
S1130AC00B01C01A5241C3088B4201D3CB00C01A98
S1130AD0524183088B4201D38B00C01A5241430810
S1130AE08B4201D34B00C01A5241884200D3401AB2
S1130AF05241CFD201461046704708B500F0E8F8DD
S1130B0008BDFEE762B6704762B6704780B5FFF76E
S1130B1087FC01BD80B5FFF78AFC02BD80B5FFF7F5
S1130B20C4FC02BD80B5FFF72CFD02BD80B5FFF704
S1130B306EFD02BD80B5FFF7EBFC002801D100205B
S1130B4001E0FFF747FD02BD80B5054800680007D6
S1130B5001D5002002E000F0EFF8012002BD000002
S1130B60D0F00F4080B5642000F0B4F801BD80B52A
S1130B7000F0BFF801BD000010B500F0F3F800F07C
S1130B80A1FB354C0120207000F04CFD00202070AA
S1130B9010BD1CB5314C6946200000F0E5FC01286D
S1130BA007D101202C49087068460178200000F024
S1130BB0F5F86946200000F0AAFD012807D10020BD
S1130BC02549087068460178200000F0E7F813BD55
S1130BD0704770B506000C001F4D2878012804D119
S1130BE02100C9B2300000F045FC2878002804D167
S1130BF02100C9B2300000F069FD00F0CBF870BDEF
S1130C0000B515480078002805D0022807D004D381
S1130C10032806D007E0402006E0082004E0002076
S1130C2002E0002000E0402080B200BD00B50A4888
S1130C300078002805D0022807D004D3032806D062
S1130C4007E0402006E0082004E0002002E0002045
S1130C5000E0402080B200BDDC000020CC30002049
S1130C6010B5002400F08DF8002800D001242000E5
S1130C70C0B210BD80B500F00CF8104810490860EF
S1130C8000201049086005210F4A11600F490860CF
S1130C9001BD00200C490860704700B50A4800688F
S1130CA0C00303D509480168491C016000BD80B533
S1130CB0FFF7F3FF0548006802BD00007FBB00009A
S1130CC014E000E018E000E010E000E060330020F1
S1130CD070470000802149001B4A11601B4A1368B9
S1130CE00B4313601A4A13681943116019490880A9
S1130CF0704710B5FFF7DBFF174C216888421AD301
S1130D0016480178002908D10121017014480168AE
S1130D10802252000A43026007E0002101700C485F
S1130D200168802252000A430260FFF7C0FF0949AC
S1130D3009884018206010BD0548016880225200CF
S1130D400A4302607047000020D0044014F10F40B1
S1130D5008F10F40B033002014330020B3330020D7
S1130D6004F10F400020B74902000A7088640200B1
S1130D704323CA5402004423CA5202008A704870B2
S1130D80704700B5AF480078002801D1002000E08A
S1130D90012000BD0020BB490870704710B50178E0
S1130DA0FF2916D100F08AF8A64C4320205C0128C4
S1130DB002D1102000F07AF84420205E012807DBDD
S1130DC00120432160544420215EE01C00F052F8CD
S1130DD010BD9C49097801294BD10178C92932D029
S1130DE0CC293FD0CF293AD0D0292FD0D12933D004
S1130DF0D2292ED0F32917D0F4290FD0F5290AD0FF
S1130E00F6290ED0FA2912D0FC2913D0FD2914D0CA
S1130E10FE2915D029E000F0B0F8C5E700F0CCF8C1
S1130E20C2E700F0A1F8BFE700F0E9F8BCE700F082
S1130E308AF8B9E700F082F8B6E700F071F8B3E792
S1130E4000F062F8B0E700F0FFF8ADE700F01CF93D
S1130E50AAE700F0E5F8A7E700F044F9A4E700F0FA
S1130E6053F9A1E700F05EF99EE7202000F01EF898
S1130E709AE7ADE780B589B2FFF7ABFE01BDF8B5DF
S1130E8004000D001700002604E020783618641CC6
S1130E90FFF7C3FD2800451E0028F6D1F6B23E60D8
S1130EA00120F2BD00206749487070476549FE2261
S1130EB0CA700871022044228852704738B5FFF77F
S1130EC0F1FF604C01252570FF20E0700020211DFA
S1130ED008702279102313430B70611D0870607928
S1130EE00870FFF78DFEA071FFF7A0FEE071FFF719
S1130EF09DFE80B2000A20726572A572082044210A
S1130F006052FFF703FE31BD10B54E4C0020207037
S1130F10FFF7C8FFFF20E07001204421605210BD9C
S1130F204848FF21C17000210171427842718171EA
S1130F30C1710172062144228152704780B500209C
S1130F40FFF7B4FF01BD3F48FF21C17073498164BD
S1130F5000210171417181710721C01C4160C01ED3
S1130F6008214422815270473649FF22CA704068E2
S1130F708864012044228852704738B50500FFF781
S1130F803FFE80B2401E6978884203DA2220FFF7D0
S1130F908DFF10E06A782B4C201D92B2A16CFFF7F4
S1130FA027FDFF20E070A06C69784018A064687881
S1130FB0401C4421605231BD70B50500FFF720FE8E
S1130FC080B2401E6978884203DA2220FFF76EFF60
S1130FD014E01C4C26004836686830606A78201D8E
S1130FE092B2A16CFFF704FDFF20E070A06C697859
S1130FF0401830606878401C4421605270BD10B5C0
S1131000104CFF21E170E21D4168A06CFFF737FF2F
S1131010207100206071A07108204421605210BD2D
S113102038B5084CFF20E070002525716571FFF785
S1131030E7FDA071E57125726572072044216052B5
S113104031BD00006433002038B50500FFF7D8FD3A
S1131050334C6A1C80B2411EA06CFFF75BFD002874
S113106003D13120FFF722FF0BE0FF20E070FFF7F0
S1131070C7FDA16C80B2401E0818A0640120442161
S1131080605231BDA733002038B50500FFF7B8FD25
S113109080B2801E6978884203DA2220FFF706FFB7
S11310A01FE01F4CFF20E07001204421605268784B
S11310B0002807D1FFF73EFD002802D13120FFF7B9
S11310C0F5FE0EE0AA1C6978A06CFFF723FD00284A
S11310D003D13120FFF7EAFE03E0A06C69784018E1
S11310E0A06431BD10B50E4C4168A06CFFF716FD2D
S11310F0002803D13120FFF7D9FE04E0FF20E0707F
S113110001204421605210BD80B5FFF751FC044812
S1131110FF21C17001214422815201BDB01E000093
S11311206433002080B53120FFF7C0FE01BD00000C
S1131130FEB507000D00140068465F490CC90CC0D9
S1131140083908385D480168090A4907490F002928
S113115005D101210A02E023DB0013400360584853
S11311606A46515CFFF776FC0190002668460780CA
S113117000E0761C3000C0B212282BD2B94F01987F
S113118069460A883100C9B204235943795C514342
S1131190FFF760FC0029ECD1019869460A88310008
S11311A0C9B204235943795C5143FFF753FC2880A7
S11311B028880028DDD02888FF21891C8842D8D2BD
S11311C02000F6B204214E43B919042200F050FB6A
S11311D0012000E00020FEBD38B5A34C20680028A3
S11311E003D5D021A14800F050FB20688021C90517
S11311F00143216020688021490501432160FFF7F4
S113120056FD0500FA352068C00105D4FFF705FC3A
S1131210FFF74DFD8542F6D231BD38B5924C2068BA
S1131220002803D5F021914800F02FFB2068904955
S1131230014021602068C74901402160FFF737FD64
S11312400500FA352068C00105D5FFF7E6FBFFF776
S11312502EFD8542F6D231BD38B5834C2068002876
S113126011D420688021090601432160FFF71FFD86
S11312700500FA352068C00205D4FFF7CEFBFFF75E
S113128016FD8542F6D231BD38B5774C206800286A
S113129010D52068400040082060FFF708FD0500D5
S11312A0FA352068C00205D5FFF7B7FBFFF7FFFC4E
S11312B08542F6D231BD0000A01E00000441064064
S11312C0409C0000FEB500273800694608800422CF
S11312D0002101A800F0DDFA9F4DA048016880229A
S11312E0D2050A430260FFF7CFFFFFF775FFFFF750
S11312F0B3FF9B4C20689B4901402160FFF7C4FF6A
S1131300FFF76AFF01AA6946FA204000FFF710FFC1
S1131310002804D1FF217831544800F0B6FA20683F
S1131320A94901402160206869460988491E0906C7
S11313300143216001A821684278521E5207520FCE
S11313400A43226021688278521ED204E0239B0360
S113135013400B4323602168C278521E1204E02319
S1131360DB0213400B4323608178042901DA80787F
S113137000E004202168C0B2401E8005C02212048F
S113138002400A4322602068802101432160380022
S113139006E08E49020092B204235343CF50401C0E
S11313A0010089B28029F4D3380006E0884902009C
S11313B092B204235343CF50401C010089B2202928
S11313C0F4D3294E30687F2188431F2101433160C3
S11313D030688021890201433160306880214902EC
S11313E00143316030687B49014031607A487B4970
S11313F008607B488021C9040160002D0BD5690079
S11314004908026880239B0313430360C800C00893
S11314107449086004E0A804C000C0087149086069
S1131420714807600020C0437049086070487149E2
S11314300860306870490140316020686F4901409C
S11314402160FFF7EAFEFFF732FC0400FA3430684B
S1131450000105D5FFF7E1FAFFF729FC8442F6D233
S1131460F7BD0000601D000000400240A81D000000
S1131470FFFFFFBFFEB506000A00002529006048F3
S1131480002802D54000400801216B461A708024D0
S11314906400564A14605B4A1368DB00DB0813607F
S11314A01368594F1F40176013688027FF031F43B9
S11314B017601368554F1F4017601768BC466B468A
S11314C01B781F04F0231B033B4067463B43136018
S11314D04F4B019611E02E00F6B20327BE43F61CD3
S11314E02F00FFB2BF07BF0FF71BBC46019F2E00A2
S11314F0F6B2BE5D6746DE556D1C2E006F463F7822
S1131500F6B2BE42E7D3C9B2002905D18004C000B7
S1131510C0084049086008E0116880239B030B431E
S11315201360C000C0083B4908601068C021090569
S113153001431160FFF7BBFB050032352B480068FF
S11315402040002805D1FFF768FAFFF7B0FB854279
S1131550F4D2F7BDFFFFFFEF67060000905006408E
S113156004400240FFDFFFFFF0B50A00002319002A
S11315708024A4001D4D2E682640002E21D0184939
S11315800968090C0907090F117023490EE01E00B0
S1131590F6B20327BE43F61C1F00FFB2BF07BF0FFE
S11315A0F61B8E5D1F00FFB2C6555B1C1E0017782C
S11315B0F6B2BE42EBD32C601848006818490860A4
S11315C001210800C0B2F0BD78FF00008040024055
S11315D080480240FFFFFFDFFFFFFF5FA448024097
S11315E01041024014410240284002403040024071
S11315F006003B0020400240FFFF7FFFF7EFFFFFA4
S1131600E107000000410240FFFFCFFFFFFFF0FFB2
S1131610084102400441024018410240084002408F
S1131620C83000201CB568466F490CC90CC0083985
S113163008386E4801686E4A0A40026001688422D4
S1131640D2050A4302606B480168090A4907490F39
S1131650002907D1012102680B02E024E4001C40A8
S11316601443046064480124644A12682240002A36
S113167000D163486A46515CFFF7ECF9E1210902A5
S1131680FFF7E8F9C01DC008C004C00C80B2C00454
S1131690C00CE021C90401435A4801605A485B491F
S11316A008605B48002101605A4A11605A4A11607F
S11316B05A49F02292020A600A68882313430B6095
S11316C057490C60C0210903016013BD70B50400C3
S11316D00D002800C0B2412803DBC221514800F0AC
S11316E0D4F82800C0B200F069F8002607E0FFF73C
S11316F094F9300080B2205C00F060F8761C300071
S11317002900C9B280B289B28842F0D370BDF8B55D
S113171007000E0044480078002816D1434C2000EE
S113172000F03CF8012837D12078002834D0207804
S1131730412831DAFFF7BBFA3D49086000203D49F2
S1131740087001203849087026E03A4C374D20785B
S11317502818401C00F022F8012813D12078401CDE
S1131760207020782978884216D13800227892B2E5
S1131770691CFFF73DF900202B4908702078307070
S113178001200AE0FFF793FA29490968643181428C
S113179002D20020244908700020F2BD00B50021C7
S11317A001221A4B1B685B0D1340002B03D0224906
S11317B00968017011000800C0B200BD10B5C0B2C4
S11317C01D490860FFF773FA04000A340F480068E3
S11317D001000902C90F002905D1FFF71EF9FFF71F
S11317E066FA8442F2D210BDA81E0000A851064039
S11317F0FFFFFFBF0442064000127A000842064081
S113180080841E0010A0064000C01FC014A0064023
S113181018A0064020A0064024A0064028A00640A8
S11318202CA00640EC1D0000B53300201833002026
S11318305C330020B43300201CA0064070B4103A7E
S113184003D378C9103A78C0FBD2530701D318C91F
S113185018C001D508C908C0D20704D30B88038077
S1131860891C801C002A01D50B78037070BC70475A
S11318708B0701D18307E1D0124205D00B78491CB4
S11318800370401C521EF9D1704780B5FFF7C5F8AC
S1131890FCE710B50400080011000200200000F06D
S11318A003F8200010BD00001206130A1A43130C9B
S11318B01A4300BF094205D0830705D00270401CBB
S11318C0491EF9D1704700001300103906D330B413
S11318D01400150010393CC0FCD230BC490700D3B9
S11318E00CC000D504C0890002D30280801C0029EA
S11318F000D502707047000080B500F005F800F0D4
S113190083F800F08FF8FCE780B500F037F880200A
S1131910C0052B490A6802430A602A490A6802433F
S11319200A6029490A68104308602848016880222F
S113193052000A43026001680222914301600820B8
S1131940C04323490A6802400A6022490A681040D9
S113195008608020800020490A6802430A601F4909
S11319600A6810430860A020C0001D490A680243A9
S11319700A601C490A681043086001BD80B5FF2055
S1131980801C194908603421184A116018490A68F2
S11319901202FBD401220A600A68D201FCD515495F
S11319A0086015490860154815490860154800681D
S11319B0000E0007000F0328F8D100F048F801BD1D
S11319C02851064030510640345106400CC00440B2
S11319D0D4F00F40D8F00F4000A0044004A004400D
S11319E010D0044014D0044004410640084106408D
S11319F0004106400443064004420640010000033F
S1131A00144006401040064080B5FEF7CDFFFFF7B6
S1131A1000F8FFF72FF9FFF779F8FFF7ADF800F0BA
S1131A2061F801BD80B5FEF7F8FFFFF736F9FFF75F
S1131A30B0F800F060F801BD1E481F49016000685D
S1131A401E481F4908601F481F490860704770B549
S1131A500022100001252B000F241C4E3168090CB4
S1131A602140491C3668360E3440012C04D018D36A
S1131A70032C0CD002D314E0154813E0154C246851
S1131A802540002D01D0124800E013000AE0124C5A
S1131A902468A407A40F002C01D1104800E013000F
S1131AA000E01300DBB2002B03D0FEF7D3FF0C4998
S1131AB0086070BD0420054020C528D920210000FD
S1131AC000200540FFFF00000820054010400640AC
S1131AD000127A000842064008430640006CDC020B
S1131AE0D800002080B501201549087000F01DF8C9
S1131AF000F001F801BD10B5FFF7B2F8012813D0CA
S1131B000F4C207801280FD1FFF7D1F80D4909684F
S1131B100D4A12688918FA2252008918884203D3A0
S1131B2000202070FEF744FF10BD80B50448007803
S1131B30012803D1FFF7BBF80349086001BD000089
S1131B40B2330020C4300020C03000200020000048
S1131B500008000004000000002800000008000045
S1131B60050000000030000000080000060000002E
S1131B7000380000000800000700000000400000DA
S1131B8000080000080000000048000000080000F1
S1131B900900000000500000000800000A000000D6
S1131BA000580000000800000B0000000060000066
S1131BB0000800000C00000000680000000800009D
S1131BC00D00000000700000000800000E0000007E
S1131BD000780000000800000F00000000800000F2
S1131BE000800000100000000000010000800000E0
S1131BF011000000008001000080000012000000BD
S1131C0000000200008000001300000000800200B9
S1131C1000800000140000000000030000800000A9
S1131C201500000000800300008000001600000082
S1131C30FFB526482649274A0392274A274B284CB2
S1131C400294284C284D0195284D294E294F009780
S1131C5003E00F780770401C491C039F8F42F8D1A2
S1131C600298984207D018781070521C5B1CF7E752
S1131C7000202070641C0198A042F9D10098B04261
S1131C8004D030782870761C6D1CF7E70023180008
S1131C9019491A4A8A4212D006E004245C430C59BA
S1131CA004255D4354515B1C154CA408A342F4D392
S1131CB01449C0B2042358430858026005E0114A8D
S1131CC0C0B20423584310580160FFBDD80000205F
S1131CD0B81E0000C01E0000C00000207C1E0000D2
S1131CE0941E0000C0300020B63300200000000025
S1131CF000000000000000000000000000000020C0
S1131D00C0000000C01E000072B6002100220023A3
S1131D100024002500260027B846B946BA46BB462B
S1131D20BC460A490A4A521A013A05DD0020042336
S1131D3008601944043AFBDA064885460648804799
S1131D400648804762B6FFF7D7FDFEE70000002093
S1131D50FF57002000580020391A0000311C0000F1
S1131D6008030202090303020A0303030B04030327
S1131D700C0404030D0504030E0504040F060404F7
S1131D8010060504110705041207050513080505C7
S1131D901408060515080705160807061708080697
S1131DA01808080719080808433A5C576F726B5CF7
S1131DB0736F6674776172655C4F70656E424C54E4
S1131DC05F5333324B31315C5461726765745C53D9
S1131DD06F757263655C41524D434D305F533332CE
S1131DE04B31315C63616E2E63000000433A5C57F3
S1131DF06F726B5C736F6674776172655C4F70654C
S1131E006E424C545F5333324B31315C54617267D0
S1131E1065745C536F757263655C41524D434D301C
S1131E205F5333324B31315C72733233322E630081
S1131E3000F00DF8002801D000BF00BF00BF00BFB4
S1131E40002000BF00BFFFF757FD00F002F801209B
S1131E50704780B500F002F801BD0000074638461F
S1131E6000F002F8FBE7000080B500BF00BF024AA3
S1131E7011001820ABBEFBE72600020000B580204D
S1131E8003490A7802430A700A780242FCD000BD72
S1131E900000024000BF00BF00BF00BFFFF7C8FF43
S1131EA00001020408102040000102040810204030
S1131EB04F70656E424C5400006CDC02040000005C
S1071EC008ED00E045
S9031E9549
